:100000000C945D000C9485000C9485000C94850084
:100010000C9485000C9485000C9485000C9485004C
:100020000C9485000C9485000C9485000C9485003C
:100030000C9485000C9485000C9485000C9485002C
:100040000C94B30C0C9485000C94230D0C94FD0CB3
:100050000C9485000C9485000C9485000C9485000C
:100060000C9485000C94850000000008000201003B
:100070000003040700000000000000000000000072
:10008000250028002B0000000000240027002A0083
:10009000040404040404040402020202020203032E
:1000A0000303030301020408102040800102040836
:1000B00010200102040810206D1411241FBECFEF80
:1000C000D8E0DEBFCDBF12E0A0E0B1E0E8EBF0E3A6
:1000D00002C005900D92AC31B107D9F722E0ACE136
:1000E000B2E001C01D92A33DB207E1F710E0CDE5FB
:1000F000D0E004C02197FE010E942E17CC35D10715
:10010000C9F70E947E110C945A180C940000FC014F
:10011000918D228D892F90E0805C9F4F821B9109E9
:100120008F739927089580E090E0892B29F00E9431
:100130003A0C81110C9400000895FF920F931F93C5
:10014000CF93DF938B01EA01DB01ED91FC910680F7
:10015000F781E02D60E070E0C8010995F82ED80124
:10016000ED91FC910084F185E02D60E070E0C80124
:100170000995182FE881F9810284F385E02D8F2DF0
:100180000F2C000C990BF7FE09C0AA27BB27A81B50
:10019000B90BA25FBE4F4C91419504C0DC01A25F38
:1001A000BE4F4C9160E070E0CE010995E881F98185
:1001B0000484F585E02D812F012E000C990B17FF8B
:1001C00009C0AA27BB27A81BB90BA25FBE4F4C9141
:1001D000419504C0DC01A25FBE4F4C9160E070E02D
:1001E000CE01DF91CF911F910F91FF900994CF9392
:1001F000DF93FC0198E081E02AB120632AB9282F1F
:1002000030E0220F232F221F330B232B09F427C0AA
:10021000000000000000000000002AB12F7C2AB975
:1002200000000000000000000000000000000000CE
:1002300000000000000000000000000000000000BE
:1002400000000000000000000000000000000000AE
:1002500000000000000000000000000027C00000B7
:10026000000000000000000000000000000000008E
:10027000000000000000000000000000000000007E
:10028000000000000000000000000000000000006E
:10029000000000000000000000000000000000005E
:1002A0000000000000002AB12F7C2AB9915059F0BB
:1002B000000000000000000000000000000000003E
:1002C0000000880F99CF00000000000000008AB1F4
:1002D00080638AB9000000000000000000000000F8
:1002E000000000000000000000000000000000000E
:1002F0008AB18F7C8AB9DF015396AF014D5C5F4FA5
:100300009D018FE399B1907381F08150D9F7128AE2
:10031000118A108A1786D90160E070E0C0E0D0E051
:1003200080E090E040E850E02DC0000000000000B8
:1003300000000000000000000000000000000000BD
:1003400000000000000000000000000000000000AD
:10035000000000000000000000000000000000009D
:1003600000000000000089B180738D934A175B077D
:1003700009F4CDCF8FE399B1907309F0C2CF8150CA
:10038000D1F7C5CF2D91222341F09A01082E02C04A
:10039000359527950A94E2F701C020E0622B179665
:1003A0002C911797222341F09A01082E02C035950F
:1003B00027950A94E2F701C020E0722B1F962C913A
:1003C0001F97222339F09A01082E02C035952795F0
:1003D0000A94E2F7C22B57962C915797222339F0B3
:1003E0009A01082E02C0359527950A94E2F7D22B80
:1003F00001968830910531F6D08BC787728B618B5F
:10040000DF91CF910895DC01ED91FC910284F38599
:10041000E02D6CE070E00994FC012189211104C0F9
:1004200092899F7381E009F080E00895FC012189A1
:10043000211105C092899F7381E09F3309F080E00C
:1004400008959B0177FF02C0295F3F4F43E0359538
:1004500027954A95E1F7FC01E20FF31F218930E06F
:10046000CB0168E070E00E940617A90102C0559513
:1004700047958A95E2F7CA0181700895FC01808949
:100480000895FC0187850895FC0114A60895FC01D8
:1004900084A50895860F971F4195FC014187089513
:1004A000860F971FFC01418708959B014423E9F0C3
:1004B00077FF02C0295F3F4F53E0359527955A9546
:1004C000E1F7FC01E20FF31FCB0168E070E00E944E
:1004D000061721E030E0A90102C0440F551F8A959C
:1004E000E2F7CA019381892B1DC077FF02C0295F03
:1004F0003F4F43E0359527954A95E1F7FC01E20F20
:10050000F31FCB0168E070E00E94061721E030E0A5
:10051000A90102C0440F551F8A95E2F7CA018095D0
:100520009381892383830895660F771FFC01E60F6B
:10053000F71F8FE7489F402D1124405846830895A8
:100540006F5F7F4F660F771FFC01E60FF71F8FE786
:10055000489F402D1124405843830895660F771F0C
:10056000860F971F4058FC01468308956F5F7F4FA9
:10057000660F771F860F971F4058FC01438308952D
:10058000FC01138280E88483858386838783808748
:100590001186128608950C94CC1760E070E00C94DC
:1005A0005D10EF92FF920F931F93CF93DF93CDB720
:1005B000DEB728970FB6F894DEBF0FBECDBF8C0113
:1005C000FC01E85BFE4F8081833440F4813408F005
:1005D00057C0882331F08034E9F06DC08F3F09F0B7
:1005E0006AC089E0F8018383148283E0858380E810
:1005F00086831782108611861286FF24F394F38671
:10060000F48640E063E0C80103960E94A80FF80159
:10061000F4A64CC080911C0298012C5D3F4F7901DB
:1006200081110CC028E0C8010396FC01D70101909C
:100630000D922A95E1F741E068E00CC088E0F901ED
:10064000DE01119601900D928A95E1F741E068E094
:10065000CE0101960E94A80FF801EF2811F4128232
:1006600007C0E65BFE4F808181708083F801828342
:1006700061E070E0C8010E945D1080931C021BC005
:10068000F801138280E8848385838683878380874B
:100690001186128682E08387848741E06AE0C80180
:1006A00003960E94A80F81E0F80184A761E070E042
:1006B000C8010E945D1028960FB6F894DEBF0FBEE9
:1006C000CDBFDF91CF911F910F91FF90EF900895D3
:1006D000CF92DF92EF92FF920F931F93CF93DF930E
:1006E000EC018B017A018C819D818130910521F093
:1006F000029709F45CC011C0DB01ED91FC91008808
:10070000F189E02DCB010995882329F082E090E062
:100710009D838C836EC11D821C82D701ED91FC915B
:10072000C284D384D801ED91FC910680F781E02D3D
:1007300060E070E0C8010995682F880F770B880B7F
:10074000990B0E94E415AB01BC01CE010E94310E51
:10075000482F60E070E0C701F6010995D701ED91DF
:10076000FC91C484D584D801ED91FC910084F1857D
:10077000E02D60E070E0C8010995682F880F770BC5
:10078000880B990B0E94E415AB01BC01CE010E94BD
:10079000310E482F60E070E0C701F601DF91CF9184
:1007A0001F910F91FF90EF90DF90CF900994DA01A5
:1007B000ED91FC910284F385E02D4F8160E070E0C3
:1007C000C7010995D701ED91FC910484F585E02DD1
:1007D000498560E070E0C7010995D801ED91FC9171
:1007E0000088F189E02DC8010995882309F404C126
:1007F0008E81D801ED91FC910284F385E02D69E0B2
:1008000070E0882309F466C0C801099581110FC101
:10081000D801ED91FC910284F385E02D68E070E051
:10082000C8010995811103C1D801ED91FC910284A1
:10083000F385E02D6BE070E0C80109958111F7C0E8
:10084000D801ED91FC910284F385E02D6AE070E01F
:10085000C80109958111EBC0D801ED91FC9102848A
:10086000F385E02D61E070E0C80109958111DFC0DA
:10087000D801ED91FC910284F385E02D60E070E0F9
:10088000C80109958111D3C0D801ED91FC91028472
:10089000F385E02D62E070E0C80109958111C7C0C1
:1008A000D801ED91FC910284F385E02D6DE070E0BC
:1008B000C80109958111BBC0D801ED91FC9102845A
:1008C000F385E02D64E070E0C80109958111AFC0A7
:1008D0001E82ADC0C8010995882351F08F8198858B
:1008E0008230910514F0019719C081E090E016C0A4
:1008F000D801ED91FC910284F385E02D68E070E071
:10090000C8010995882369F02F81388589859A85E2
:1009100001972817390714F4C901019698878F8326
:1009200068C0D801ED91FC910284F385E02D6AE066
:1009300070E0C8010995882361F029853A858F8187
:1009400098850196821793070CF051C0C901019751
:100950004EC0D801ED91FC910284F385E02D6BE04F
:1009600070E0C8010995882351F089859A858435FE
:10097000910514F401963BC08FE390E038C0D80194
:10098000ED91FC910284F385E02D64E070E0C801F4
:1009900009958823D1F08B81813049F0823071F044
:1009A00087E190E098878F8385E290E020C084E122
:1009B00090E098878F8380E290E019C08EE190E00C
:1009C00098878F8389E290E012C0D801ED91FC9165
:1009D0000284F385E02D6DE070E0C801099588235D
:1009E00031F188E090E098878F838BE190E09A87DF
:1009F000898781E08E831BC08091CB029091CC02CD
:100A0000009799F06F810E948E0A8091CB0290919D
:100A1000CC02698501960E948E0A8091CB0290914A
:100A2000CC026B8102960E948E0A1D821C82DF918D
:100A3000CF911F910F91FF90EF90DF90CF9008958D
:100A4000FC01848DDF01A80FB11DA35ABF4F2C916B
:100A5000848D90E001968F739927848FA689B7893A
:100A60002C93A089B1898C91837080648C93938D31
:100A7000848D981306C00288F389E02D80818F7DD4
:100A80008083089508950F931F93CF93DF93EC0114
:100A90001A828CE091E0998388831B820091CB02BB
:100AA0001091CC0201151105F1F581E00E94E00DD5
:100AB0008C019093CC028093CB02892BA1F563E04B
:100AC00070E081E00E94550D9093CC028093CB02A0
:100AD0001B8227E130E03E872D8725E230E03C870E
:100AE0002B8727E430E0388B2F8728E030E03887E9
:100AF0002F832BE130E03A872987009731F168E0B6
:100B00000E948E0A8091CB029091CC026985019659
:100B10000E948E0A8091CB029091CC026B8102964A
:100B20000E948E0A12C0C8010E94B21490E09887F9
:100B30008F83C80101960E94B21490E09A8789873A
:100B4000C80102960E94B2148B838B81813069F0B8
:100B50008230B1F087E190E09E878D8785E290E05A
:100B60009C878B8787E490E015C084E190E09E87A6
:100B70008D8780E290E09C878B8785E390E00AC0B8
:100B80008EE190E09E878D8789E290E09C878B873D
:100B900089E490E0988B8F8781E090E09D838C833F
:100BA000DF91CF911F910F910895CF92DF92EF9235
:100BB000FF920F931F93CF93DF93EB018A01DA012A
:100BC000ED91FC91C088D188E881F9810284F38598
:100BD000E02D6BE070E0CE010995F82EE881F981F7
:100BE0000284F385E02D6DE070E0CE0109954F2D74
:100BF000481B61E070E0C801F6010995D801ED914C
:100C0000FC91E688F788E881F9810284F385E02D7C
:100C100064E070E0CE010995482F64E070E0C801FF
:100C2000F7010995D801ED91FC91E688F788E881F4
:100C3000F9810284F385E02D6AE070E0CE01099528
:100C4000482F6CE070E0C801F7010995D801ED91DB
:100C5000FC91E688F788E881F9810284F385E02D2C
:100C600069E070E0CE010995482F63E070E0C801AB
:100C7000F7010995D801ED91FC91E688F788E881A4
:100C8000F9810284F385E02D68E070E0CE010995DA
:100C9000482F62E070E0C801F7010995D801ED9195
:100CA000FC91E688F788E881F9810284F385E02DDC
:100CB00066E070E0CE010995482F61E070E0C80160
:100CC000F7010995D801ED91FC91E688F788E88154
:100CD000F9810284F385E02D67E070E0CE0109958B
:100CE000482F60E070E0C801F7010995D801ED9147
:100CF000FC91E688F788E881F9810284F385E02D8C
:100D00006CE070E0CE010995482F6DE070E0C801FD
:100D1000F7010995D801ED91FC91E688F788E88103
:100D2000F9810284F385E02D65E070E0CE0109953C
:100D3000482F6EE070E0C801F7010995D801ED91E8
:100D4000FC91E688F788E881F9810284F385E02D3B
:100D500063E070E0CE010995482F6BE070E0C801B8
:100D6000F7010995D801ED91FC91E688F788E881B3
:100D7000F9810284F385E02D62E070E0CE010995EF
:100D8000482F6AE070E0C801F7010995D801ED919C
:100D9000FC91E688F788E881F9810284F385E02DEB
:100DA00061E070E0CE010995482F68E070E0C8016D
:100DB000F7010995D801ED91FC91E688F788E88163
:100DC000F9810284F385E02D60E070E0CE010995A1
:100DD000482F69E070E0C801F701DF91CF911F91C2
:100DE0000F91FF90EF90DF90CF900994CF92DF9218
:100DF000EF92FF920F931F93CF93DF93EB018A0142
:100E0000DA01ED91FC91C684D784E881F9810284EE
:100E1000F385E02D68E070E0CE010995F82EE881B9
:100E2000F9810284F385E02D69E070E0CE01099537
:100E30004F2D481B61E070E0C801F6010995D8010B
:100E4000ED91FC91C088D188E881F9810284F38515
:100E5000E02D6BE070E0CE010995F82EE881F98174
:100E60000284F385E02D6AE070E0CE0109954F2DF4
:100E7000481B61E070E0C801F6010995D801ED91C9
:100E8000FC91E688F788E881F9810284F385E02DFA
:100E900064E070E0CE010995482F64E070E0C8017D
:100EA000F7010995D801ED91FC91E688F788E88172
:100EB000F9810284F385E02D65E070E0CE010995AB
:100EC000482F6CE070E0C801F7010995D801ED9159
:100ED000FC91E688F788E881F9810284F385E02DAA
:100EE00066E070E0CE010995482F61E070E0C8012E
:100EF000F7010995D801ED91FC91E688F788E88122
:100F0000F9810284F385E02D67E070E0CE01099558
:100F1000482F60E070E0C801F7010995D801ED9114
:100F2000FC91E688F788E881F9810284F385E02D59
:100F30006CE070E0CE010995482F6DE070E0C801CB
:100F4000F7010995D801ED91FC91E688F788E881D1
:100F5000F9810284F385E02D6DE070E0CE01099502
:100F6000482F6EE070E0C801F7010995D801ED91B6
:100F7000FC91E688F788E881F9810284F385E02D09
:100F800063E070E0CE010995482F6BE070E0C80186
:100F9000F7010995D801ED91FC91E688F788E88181
:100FA000F9810284F385E02D62E070E0CE010995BD
:100FB000482F6AE070E0C801F7010995D801ED916A
:100FC000FC91E688F788E881F9810284F385E02DB9
:100FD00061E070E0CE010995482F68E070E0C8013B
:100FE000F7010995D801ED91FC91E688F788E88131
:100FF000F9810284F385E02D60E070E0CE0109956F
:10100000482F69E070E0C801F701DF91CF911F918F
:101010000F91FF90EF90DF90CF900994CF92DF92E5
:10102000EF92FF920F931F93CF93DF93EB018A010F
:10103000DA01ED91FC91C684D784E881F9810284BC
:10104000F385E02D68E070E0CE010995F82EE88187
:10105000F9810284F385E02D69E070E0CE01099505
:101060004F2D481B61E070E0C801F6010995D801D9
:10107000ED91FC91C088D188E881F9810284F385E3
:10108000E02D6BE070E0CE010995F82EE881F98142
:101090000284F385E02D6AE070E0CE0109954F2DC2
:1010A000481B61E070E0C801F6010995D801ED9197
:1010B000FC91E688F788E881F9810284F385E02DC8
:1010C00064E070E0CE010995482F64E070E0C8014B
:1010D000F7010995D801ED91FC91E688F788E88140
:1010E000F9810284F385E02D6DE070E0CE01099571
:1010F000482F6CE070E0C801F7010995D801ED9127
:10110000FC91E688F788E881F9810284F385E02D77
:1011100066E070E0CE010995482F61E070E0C801FB
:10112000F7010995D801ED91FC91E688F788E881EF
:10113000F9810284F385E02D67E070E0CE01099526
:10114000482F60E070E0C801F7010995D801ED91E2
:10115000FC91E688F788E881F9810284F385E02D27
:101160006CE070E0CE010995482F6DE070E0C80199
:10117000F7010995D801ED91FC91E688F788E8819F
:10118000F9810284F385E02D65E070E0CE010995D8
:10119000482F6EE070E0C801F7010995D801ED9184
:1011A000FC91E688F788E881F9810284F385E02DD7
:1011B00063E070E0CE010995482F6BE070E0C80154
:1011C000F7010995D801ED91FC91E688F788E8814F
:1011D000F9810284F385E02D62E070E0CE0109958B
:1011E000482F6AE070E0C801F7010995D801ED9138
:1011F000FC91E688F788E881F9810284F385E02D87
:1012000061E070E0CE010995482F68E070E0C80108
:10121000F7010995D801ED91FC91E688F788E881FE
:10122000F9810284F385E02D60E070E0CE0109953C
:10123000482F69E070E0C801F701DF91CF911F915D
:101240000F91FF90EF90DF90CF9009944F925F92B3
:101250006F927F928F929F92AF92BF92CF92DF92C6
:10126000EF92FF92CF93DF937B01EA01DB01ED91D7
:10127000FC910680F781E02D60E070E0C7010995E0
:10128000682F880F770B880B990B0E94E4154B0190
:101290005C01D701ED91FC910084F185E02D60E0C7
:1012A00070E0C7010995682F880F770B880B990BA1
:1012B0000E94E4156B017C0120E030E04AEA52E430
:1012C000C501B4010E943A1520E030E048EC52E438
:1012D0000E9499162B013C0120E030E0A9010E94F8
:1012E000351587FF11C020E030E04AEA52E4C5011D
:1012F000B40190580E943A1520E030E048EC52E4E6
:101300000E9499162B013C0120E030E0A901C501A3
:10131000B4010E94351520E030E0A901882379F05E
:10132000C501B4010E94351587FD05C020E030E0FD
:1013300040E85FE304C020E030E040E85FEBC30139
:10134000B2010E9499164B015C0120E030E04AEAAC
:1013500052E4C701B6010E943A1520E030E048ECA3
:1013600052E40E9499162B013C0120E030E0A901D3
:101370000E94351587FF11C020E030E04AEA52E4B0
:10138000C701B60190580E943A1520E030E048ECC1
:1013900052E40E9499162B013C0120E030E0A901A3
:1013A000C701B6010E94351520E030E0A90188236D
:1013B00079F0C701B6010E94351587FD05C020E010
:1013C00030E040E85FE304C020E030E040E85FEB5D
:1013D000C301B2010E9499166B017C0120E030E04C
:1013E00040E053ECC501B4010E94351587FD11C0E2
:1013F00020E030E040E053E4C501B4010E949416BF
:1014000087FD0CC0812C912C3EEFA32E32E4B32E2D
:1014100005C0812C912CA12C23ECB22E20E030E0D1
:1014200040E053ECC701B6010E94351587FD11C09D
:1014300020E030E040E053E4C701B6010E9494167A
:1014400087FD0CC0C12CD12C9EEFE92E92E4F92E21
:1014500005C0C12CD12CE12C83ECF82EC501B401C0
:101460000E94AC15462FE881F9810284F385E02DB6
:1014700060E070E0CE010995C701B6010E94AC158D
:10148000462FE881F9810484F585E02D60E070E065
:10149000CE01DF91CF91FF90EF90DF90CF90BF9082
:1014A000AF909F908F907F906F905F904F90099436
:1014B000EF92FF920F931F93CF93DF938B01EA017B
:1014C000E881F981E284F384DB01ED91FC910680EF
:1014D000F781E02D60E070E0C8010995482F60E0D9
:1014E00070E0CE01F7010995E881F981E484F58483
:1014F000D801ED91FC910084F185E02D60E070E071
:10150000C8010995482F60E070E0CE01F701DF9136
:10151000CF911F910F91FF90EF9009940F931F931C
:10152000CF938C01C62F0E94B214C81721F06C2FE4
:10153000C8010E94BA148C2FCF911F910F9108956A
:101540002091CD023091CE022115310529F0682F6E
:10155000C90101960C948E0A0895682F8091CD02DE
:101560009091CE02009711F00C948E0A089580910C
:10157000CD029091CE02892BF9F480E00E94E00D1B
:101580009093CE028093CD02892BB1F462E070E09B
:1015900080E00E94550D9093CE028093CD0200977B
:1015A00059F063E00E948E0A8091CD029091CE02A4
:1015B00062E001960C948E0A08950F931F93CF93C7
:1015C000DF938C01EB01FC018381E881F9818823A1
:1015D00059F00684F785E02DCB010995882309F49D
:1015E000E3C0F8011382E0C00284F385E02D64E0DB
:1015F00070E0CE010995882381F083E090E00E949D
:101600003417FC0112822FEE31E031832083BC01BC
:10161000CE010E94160E80E017C0E881F981028495
:10162000F385E02D66E070E0CE010995882391F006
:1016300081E190E00E9434178C010E944305B801BB
:10164000CE010E94160E83E0DF91CF911F910F9182
:101650000C94AD0AE881F9810284F385E02D67E0FE
:1016600070E0CE010995882381F083E090E00E942C
:101670003417FC01128225EF31E031832083BC0155
:10168000CE010E94160E82E0DFCFE881F98102844C
:10169000F385E02D6BE070E0CE010995882381F0A1
:1016A00083E090E00E943417FC0112822BEF31E0BE
:1016B00031832083BC01CE010E94160E81E0C4CF8D
:1016C000E881F9810284F385E02D62E070E0CE01CB
:1016D00009958823D1F082E090E00E9434178C01B4
:1016E00089EE91E0F801918380838C819D81009740
:1016F00011F00E94CC171D830C838E819F819B83E8
:101700008A831F821E8281E049C0E881F9810284B8
:10171000F385E02D60E070E0CE0109958823D1F0DB
:1017200082E090E00E9434178C0183EE91E0F80192
:10173000918380838C819D81009711F00E94CC174A
:101740001D830C838E819F819B838A831F821E82CF
:1017500082E024C0E881F9810284F385E02D65E010
:1017600070E0CE0109958823F9F082E090E00E94B4
:1017700034178C018DED91E0F801918380838C8189
:101780009D81009711F00E94CC171D830C838E81E0
:101790009F819B838A831F821E8280E0DF91CF918D
:1017A0001F910F910C94A00ADF91CF911F910F917F
:1017B0000895CF92DF92EF92FF920F931F93CF93F2
:1017C000DF936C017A018B01C0E0D0E0CE15DF051C
:1017D00081F0D8016D918D01D601ED91FC910190C0
:1017E000F081E02DC6010995892B11F02196EECFED
:1017F0007E01C701DF91CF911F910F91FF90EF9074
:10180000DF90CF900895089580E090E00895FC0166
:10181000538D448D252F30E0842F90E0821B930B55
:10182000541710F0CF96089501970895FC01918DFB
:10183000828D981761F0828DDF01A80FB11D5D9632
:101840008C91928D9F5F9F73928F90E008958FEFA0
:101850009FEF0895FC01918D828D981731F0828D54
:10186000E80FF11D858D90E008958FEF9FEF0895AB
:101870000E9455188EE292E00E94870021E0892B99
:1018800009F420E0822F0895EF92FF920F931F93A7
:10189000CF93DF93EC0181E0888F9B8D8C8D981323
:1018A00005C0E889F989808185FD26C0F62E0B8D5B
:1018B00010E00F5F1F4F0F731127E02E8C8DE81281
:1018C0000CC00FB607FCFACFE889F989808185FF43
:1018D000F5CFCE010E942005F1CF8B8DFE01E80FE0
:1018E000F11DE35AFF4FF0829FB7F8940B8FEA89FE
:1018F000FB89808180620AC09FB7F894EE89FF89D6
:101900006083E889F98980818370806480839FBFC8
:1019100081E090E0DF91CF911F910F91FF90EF90C8
:101920000895CF93DF93EC01888D8823C9F0EA896D
:10193000FB89808185FD05C0A889B9898C9186FDC8
:101940000FC00FB607FCF5CF808185FFF2CFA889C5
:10195000B9898C9185FFEDCFCE010E942005E7CF9C
:10196000DF91CF9108951F920F920FB60F9211241D
:101970002F933F938F939F93AF93BF9380912302B5
:1019800090912402A0912502B0912602309122026A
:1019900023E0230F2D3720F40196A11DB11D05C0B2
:1019A00026E8230F0296A11DB11D209322028093E9
:1019B000230290932402A0932502B09326028091E3
:1019C000270290912802A0912902B0912A02019643
:1019D000A11DB11D8093270290932802A093290294
:1019E000B0932A02BF91AF919F918F913F912F9118
:1019F0000F900FBE0F901F9018951F920F920FB669
:101A00000F9211242F933F934F935F936F937F9384
:101A10008F939F93AF93BF93EF93FF938EE292E0E8
:101A20000E942005FF91EF91BF91AF919F918F91FF
:101A30007F916F915F914F913F912F910F900FBECA
:101A40000F901F9018951F920F920FB60F921124AE
:101A50002F938F939F93EF93FF93E0913E02F0912A
:101A60003F028081E0914402F091450282FD12C064
:101A70009081809147028F5F8F7320914802821777
:101A800051F0E0914702F0E0E25DFD4F958F8093C9
:101A9000470201C08081FF91EF919F918F912F911B
:101AA0000F900FBE0F901F9018958F929F92AF923C
:101AB000BF92CF92DF92EF92FF920F931F93CF933B
:101AC000DF93C82E5B01E0902C02F0902D02C0E065
:101AD000D0E00AE010E0EC16FD060CF462C0C8018C
:101AE0000E94B21498012E5F3F4F49018F3F21F0B1
:101AF000EC16FD0609F04CC0C4010E94B214D82EA9
:101B0000EC16FD0651F090E08A159B050CF440C0E0
:101B10009C2F8D2FE701E92EF82E6C2DC8010E9415
:101B20008E0A60E0C80101960E948E0A0D5F1F4F69
:101B3000EC16FD06A1F08D2D90E00297A816B906CF
:101B40008CF47801EA0CFB1C6FEFC7010E948E0A2F
:101B50006D2D6A196350C70102960E948E0A219664
:101B60006A2D01C06D2DC4010E948E0A80912C0245
:101B700090912D028C179D0749F0D0932D02C093B0
:101B80002C026C2F81E090E00E948E0AC8010BC0ED
:101B9000C4010E94B21490E00396080F191F219609
:101BA0009ACF80E090E0DF91CF911F910F91FF904D
:101BB000EF90DF90CF90BF90AF909F908F9008955F
:101BC000DF92EF92FF920F931F93CF93DF93D82E64
:101BD000E0902C02F0902D0200E010E0CAE0D0E08E
:101BE0000E151F05CCF4CE010E94B214D81209C004
:101BF000CE0101960E94B214811103C0CE0103965A
:101C00000DC0CE0102960E94B21490E00396C80F58
:101C1000D91F0F5F1F4FE4CF80E090E0DF91CF919D
:101C20001F910F91FF90EF90DF9008950F931F93F6
:101C3000CF93DF93EC018B018E819F81009721F080
:101C40000E94CC171F821E828A819B81009711F00F
:101C50000E94CC171B830A83DF91CF911F910F91B4
:101C600008952F923F924F925F926F927F928F9240
:101C70009F92AF92BF92CF92DF92EF92FF920F931B
:101C80001F93CF93DF93CDB7DEB728970FB6F894A5
:101C9000DEBF0FBECDBF9E838D836A017B0120E036
:101CA00030E040E053E4C701B6010E9494161816D4
:101CB00054F420E030E040E853E4C701B6010E944C
:101CC000C8146B017C0120E030E0A901C701B60116
:101CD0000E94351587FF0BC0F7FAF094F7F8F094DF
:101CE000812C912C90E8A92E9FEBB92E13C020E0F7
:101CF00030E0A901C701B6010E943515882339F0EB
:101D0000812C912C80E8A82E8FE3B82E03C0812C63
:101D1000912C5401ED81FE8127803084B101032C88
:101D2000000C880B990B0E94E4152B013C01A701C4
:101D300096010E943515ED81FE8118160CF4BCC089
:101D400001851285B801012E000C880B990B0E94A9
:101D5000E41569837A838B839C83A70196010E9493
:101D6000941618160CF041C0ED81FE810584F685AD
:101D7000E02DFA83E983ED81FE81638574852981F5
:101D80003A81621B730B072E000C880B990B0E9483
:101D9000E4156D837E838F839887A3019201C70129
:101DA000B6010E94C8149B01AC016D817E818F81B8
:101DB00098850E9499166B017C01B801621973091C
:101DC000072E000C880B990B0E94E4159B01AC01B7
:101DD000C701B6010E943A156B017C01E981FA81C5
:101DE000BF01FF0F880B990B45C020E030E04AEAA5
:101DF00052E4C701B6010E94351587FF42C0ED814C
:101E0000FE810384F485E02DFE83ED8360E470E0C1
:101E10006E1B7F0B072E000C880B990B0E94E4159C
:101E20002B013C0129813A814B815C81C701B601BC
:101E30000E94C8149B01AC01C301B2010E94991613
:101E40006B017C0165E570E0601B710B072E000CD7
:101E5000880B990B0E94E4159B01AC01C701B601E8
:101E60000E943A156B017C012D813E81B901330F2F
:101E7000880B990B0E94E4159B01AC01C701B601C8
:101E800018C020E030E04AEA52E4C701B6010E94DF
:101E9000C81420E030E04CE752E40E94991620E09C
:101EA00030E048E252E40E943A1520E030E040E899
:101EB00052E40E94C91410C065857685072E000C77
:101EC000880B990B0E94E415A70196010E949916B0
:101ED000A30192010E943A15A50194010E9499164E
:101EE0006B017C0120E030E040E053EC0E943515AE
:101EF00087FD10C020E030E04EEF52E4C701B6018C
:101F00000E94941618164CF0C701B6010E94AC1539
:101F1000CB0105C080E89FEF02C08FE790E02896D4
:101F20000FB6F894DEBF0FBECDBFDF91CF911F91EA
:101F30000F91FF90EF90DF90CF90BF90AF909F9068
:101F40008F907F906F905F904F903F902F9008956B
:101F5000FC0128E0539A808190E0880F892F881F28
:101F6000990B892B09F430C000000000000000002C
:101F70000000000000000000539800000000000076
:101F80000000000000000000000000000000000051
:101F90000000000000000000000000000000000041
:101FA0000000000000000000000000000000000031
:101FB0000000000000000000000000000000000021
:101FC00000000000000030C0000000000000000021
:101FD0000000000000000000000000000000000001
:101FE00000000000000000000000000000000000F1
:101FF00000000000000000000000000000000000E1
:1020000000000000000000000000000000000000D0
:1020100000000000000000000000000000000000C0
:102020000000000000005398215069F000000000FB
:10203000000000000000000000000000000080819F
:10204000880F808387CF00000000000000006150EF
:1020500031F0000000000000000031967ACF00004F
:102060000000000000000000000000000000539A83
:102070000000000000000000000000000000000060
:1020800000000000000000000000000000004423E9
:1020900091F00000000000000000000000000000BF
:1020A0000000000000000000000000000000000030
:1020B00000000000000053980895CF93DF93DC01E7
:1020C000FC01E85BFE4F83E0EF0119928A95E9F786
:1020D000EF01161617069CF484EC99E04B9907C0A3
:1020E00081E09C968C939C9728E030E01BC0019780
:1020F000A9F79C968C919C97882309F461C09C96C3
:102100008C919C9781110AC080E290E04B9902C0AB
:1021100080E290E0019718161906C4F328E030E039
:102120004B99FECF000000000000000000000000FE
:10213000000000000000000000000000000000009F
:10214000000000000000000000000000000000008F
:10215000000000000000000000000000000000007F
:10216000000000000000000000000000000000006F
:102170004B9B03C08081816080832150310931F005
:102180008081880F80834B9BFECFCACF88818034AB
:1021900041F4CD01865B9E4FE817F90711F03196A7
:1021A000BDCF4B9BFECF8CE090E04B9902C08CE002
:1021B00090E0019718161906C4F381E090E002C080
:1021C00080E090E0DF91CF910895CF93DF9390E08E
:1021D000FC01EC55FF4F2491FC01E057FF4F849127
:1021E0008823C1F090E0880F991FFC01EA57FF4F48
:1021F000C591D491FC01E458FF4FA591B4919FB7CC
:10220000F8948881E22FE0958E2388838C91E823CF
:10221000EC939FBFDF91CF91089590E0FC01E859C6
:10222000FF4F2491FC01EC55FF4F3491FC01E05726
:10223000FF4FE491EE23B9F1222339F1233091F0DD
:1022400038F42130A9F0223001F584B58F7D12C019
:10225000273091F02830A1F02430B9F4809180002B
:102260008F7D03C0809180008F77809380000DC0A8
:1022700084B58F7784BD09C08091B0008F7703C08B
:102280008091B0008F7D8093B000F0E0EE0FFF1FD3
:10229000E458FF4FA591B4919FB7F8948C91309575
:1022A00038233C939FBF0895682F8EE292E00C94F0
:1022B000440C3FB7F8948091270290912802A09196
:1022C0002902B0912A0226B5A89B05C02F3F19F01C
:1022D0000196A11DB11D3FBFBA2FA92F982F8827A6
:1022E000820F911DA11DB11DBC01CD0142E0660F01
:1022F000771F881F991F4A95D1F70895CF93DF93D1
:1023000000D01F92CDB7DEB7789484B5826084BDCB
:1023100084B5816084BD85B5826085BD85B58160E9
:1023200085BD80916E00816080936E001092810067
:102330008091810082608093810080918100816022
:1023400080938100809180008160809380008091E3
:10235000B10084608093B1008091B000816080936F
:10236000B00080917A00846080937A0080917A0036
:10237000826080937A0080917A00816080937A00F5
:1023800080917A00806880937A001092C100E09179
:102390003E02F0913F0282E08083E0913A02F091A8
:1023A0003B021082E0913C02F0913D0280E180838B
:1023B00010924602E0914202F091430286E080834F
:1023C000E0914002F0914102808180618083E09140
:1023D0004002F0914102808188608083E091400258
:1023E000F0914102808180688083E0914002F09109
:1023F000410280818F7D8083809100019091010155
:102400000197909301018093000143E050E062E066
:1024100070E0CE0101960E94A2148981853A31F4C0
:102420008A818E3919F48B818C3811F080E04DC08F
:1024300089E090E00E94B2148233A1F162E389E066
:1024400090E00E948E0A10922D0210922C0260E001
:1024500080E090E00E948E0A60912C0281E090E082
:102460000E948E0A80918E0190918F01A09190011F
:1024700089839A83AB83CE0101967C0102E010E050
:10248000D701DD907D01C8010E94B214D81621F059
:102490006D2DC8010E94BA140F5F1F4F0530110542
:1024A00079F712C080E090E00E94B21490E090931F
:1024B0002D0280932C0281E090E00E94B21490E003
:1024C00090932D0280932C0281E0809321028BE473
:1024D00091E00E9434178C0185E991E0F801918325
:1024E0008083339651E2F52EDF012F2D1D922A9520
:1024F000E9F7EB5BFE4F83E0DF011D928A95E9F778
:10250000F80114A61093200200931F0284E390E0C8
:102510000E943417FC0187EC91E091838083178639
:10252000108A118A128ACF014396DC011D92FA9417
:10253000E9F79587848780E290E093878287168603
:10254000F0931E02E0931D0283E00E940D1183E0D0
:102550000E94E510F80112820E94B70A8091CD0214
:102560009091CE020097C1F001960E94B214813082
:1025700049F0823089F082E090E00E9434172DED1E
:1025800031E010C082E090E00E94341729EE31E083
:10259000FC013183208309C082E090E00E9434175F
:1025A00023EE31E0DC012D933C936C010E94B70ACD
:1025B0008091CD029091CE020097F9F00E94B21462
:1025C0008230D9F0833021F1813049F083E090E00E
:1025D0000E943417FC0112822FEE31E016C083E016
:1025E00090E00E943417DC0112961C9212972BEF98
:1025F00031E02D933C938C0112C083E090E00E9467
:102600003417FC01128225EF31E031832083F3CFB0
:1026100081E190E00E9434178C010E944305A09054
:102620001F02B0902002E0901D02F0901E0285E093
:102630000E940D1185E00E94E51084E00E940D11BA
:1026400084E00E94E510D7011996BC92AE921897CB
:1026500012960C93129713961C9313971496CC9280
:1026600014971596DC92159717961C921E92169742
:1026700031E0632E32E0732E5524539448E0242E2B
:10268000312C80912102882309F41CC180911F0202
:1026900090912002DC01ED91FC910190F081E02D00
:1026A00009958111F7C000911D0210911E02F801D9
:1026B0008685C484D584A284B384882351F1E12C17
:1026C000F12CEA14FB0464F5C701F7FC079623E03C
:1026D000959587952A95E1F7F601E80FF91F208176
:1026E000022E000C330BC701B1010E94061702C075
:1026F000359527958A95E2F7C9018170992720FFC2
:1027000002C081E390E00E945411FFEFEF1AFF0A2C
:10271000D8CF7601C7018C199D098A159B057CF0DD
:102720008AE090E00E945411D801ED91FC9104845C
:10273000F585E02DC801099581110EC038C0F7015B
:1027400081917F01882319F081E390E002C080E04D
:1027500090E00E945411DECFD8011296ED91FC91C9
:102760001397309719F08281811121C084E090E0A5
:102770000E9434177C01FC01718260825382528274
:10278000892B09F4A2C0F80186819781009711F086
:102790000E94CC17D80112968D919C911397179691
:1027A0009C938E9316971396FC92EE921297C0907C
:1027B0000001D09001010D2C000CEE08FF080E94D2
:1027C00059114B015C01C114D104E104F104F1F091
:1027D0000E945911DC01CB0188199909AA09BB098A
:1027E000883E9340A105B10570F3F1E0CF1AD108FE
:1027F000E108F10828EE820E23E0921EA11CB11C14
:10280000C114D104E104F10419F7DDCFF89400916B
:102810001D0210911E02D801ED91FC910480F581FA
:10282000E02DC8010995F80180859185DC01ED91C5
:10283000FC910084F185E02D0995F8018281938156
:10284000009751F040855185DC01ED91FC9101909C
:10285000F081E02DB8010995F80186819781892BD7
:1028600071F484819581009751F040855185DC0198
:10287000ED91FC910190F081E02DB80109958091D6
:102880001F0290912002DC01ED91FC910480F58102
:10289000E02D099580911F0290912002DC01ED91BD
:1028A000FC910280F381E02D0995F89480911F023C
:1028B00090912002DC01ED91FC910680F781E02DE2
:1028C000099578940E949300DCCEF8018681978167
:1028D00093838283178216826ACFEEE2F2E013823C
:1028E000128288EE93E0A0E0B0E084839583A68313
:1028F000B7838DE092E09183808385EC90E09587AB
:10290000848784EC90E09787868780EC90E0918BB9
:10291000808B81EC90E0938B828B82EC90E0958BA6
:10292000848B86EC90E0978B868B118E128E138EA3
:10293000148E1092CC021092CB021092CE02109202
:10294000CD020895DC01CB01FC01F999FECF06C050
:10295000F2BDE1BDF89A319600B40D92415050405D
:10296000B8F70895F999FECF92BD81BDF89A9927DD
:1029700080B50895262FF999FECF1FBA92BD81BD6B
:1029800020BD0FB6F894FA9AF99A0FBE01960895F1
:102990005058BB27AA270E94E0140C945A160E9494
:1029A0004C1638F00E94531620F039F49F3F19F46A
:1029B00026F40C9449160EF4E095E7FB0C944316AC
:1029C000E92F0E946B1658F3BA1762077307840742
:1029D000950720F079F4A6F50C948D160EF4E09589
:1029E0000B2EBA2FA02D0B01B90190010C01CA01C9
:1029F000A0011124FF27591B99F0593F50F4503E74
:102A000068F11A16F040A22F232F342F4427585F65
:102A1000F3CF469537952795A795F0405395C9F77D
:102A20007EF41F16BA0B620B730B840BBAF0915035
:102A3000A1F0FF0FBB1F661F771F881FC2F70EC0D4
:102A4000BA0F621F731F841F48F4879577956795A7
:102A5000B795F7959E3F08F0B0CF9395880F08F093
:102A60009927EE0F9795879508950E941F1608F4F1
:102A700081E008950E944E150C945A160E94531638
:102A800058F00E944C1640F029F45F3F29F00C9456
:102A9000431651110C948E160C9449160E946B1615
:102AA00068F39923B1F3552391F3951B550BBB277D
:102AB000AA2762177307840738F09F5F5F4F220FC2
:102AC000331F441FAA1FA9F335D00E2E3AF0E0E8B9
:102AD00032D091505040E695001CCAF72BD0FE2F03
:102AE00029D0660F771F881FBB1F26173707480797
:102AF000AB07B0E809F0BB0B802DBF01FF2793584F
:102B00005F4F3AF09E3F510578F00C9443160C94B9
:102B10008E165F3FE4F3983ED4F3869577956795DC
:102B2000B795F7959F5FC9F7880F911D9695879583
:102B300097F90895E1E0660F771F881FBB1F6217A2
:102B400073078407BA0720F0621B730B840BBA0B60
:102B5000EE1F88F7E09508950E94B3156894B111AF
:102B60000C948E1608950E94731688F09F5798F063
:102B7000B92F9927B751B0F0E1F0660F771F881F82
:102B8000991F1AF0BA95C9F714C0B13091F00E949C
:102B90008D16B1E008950C948D16672F782F882735
:102BA000B85F39F0B93FCCF3869577956795B395C3
:102BB000D9F73EF490958095709561957F4F8F4F32
:102BC0009F4F0895E89409C097FB3EF49095809537
:102BD000709561957F4F8F4F9F4F9923A9F0F92FE3
:102BE00096E9BB279395F695879577956795B79561
:102BF000F111F8CFFAF4BB0F11F460FF1BC06F5F47
:102C00007F4F8F4F9F4F16C0882311F096E911C058
:102C1000772321F09EE8872F762F05C0662371F079
:102C200096E8862F70E060E02AF09A95660F771F8D
:102C3000881FDAF7880F9695879597F90895990F69
:102C40000008550FAA0BE0E8FEEF16161706E80776
:102C5000F907C0F012161306E407F50798F0621B97
:102C6000730B840B950B39F40A2661F0232B242B6C
:102C7000252B21F408950A2609F4A140A6958FEF8B
:102C8000811D811D089597F99F6780E870E060E0DD
:102C900008959FEF80EC089500240A9416161706F5
:102CA00018060906089500240A941216130614063D
:102CB00005060895092E0394000C11F4882352F0A0
:102CC000BB0F40F4BF2B11F460FF04C06F5F7F4F58
:102CD0008F4F9F4F089557FD9058440F551F59F03F
:102CE0005F3F71F04795880F97FB991F61F09F3FF9
:102CF00079F087950895121613061406551FF2CF22
:102D00004695F1DF08C0161617061806991FF1CF71
:102D100086957105610508940895E894BB27662798
:102D20007727CB0197F908950E941F1608F48FEFBB
:102D300008950E94AC160C945A160E944C1638F056
:102D40000E94531620F0952311F00C9443160C9416
:102D5000491611240C948E160E946B1670F3959FE1
:102D6000C1F3950F50E0551F629FF001729FBB2782
:102D7000F00DB11D639FAA27F00DB11DAA1F649F1E
:102D80006627B00DA11D661F829F2227B00DA11DD1
:102D9000621F739FB00DA11D621F839FA00D611D57
:102DA000221F749F3327A00D611D231F849F600D78
:102DB000211D822F762F6A2F11249F5750409AF0A1
:102DC000F1F088234AF0EE0FFF1FBB1F661F771F2D
:102DD000881F91505040A9F79E3F510580F00C94F8
:102DE00043160C948E165F3FE4F3983ED4F3869519
:102DF00077956795B795F795E7959F5FC1F7FE2B98
:102E0000880F911D9695879597F9089597FB072E42
:102E100016F4009407D077FD09D00E941A1707FC1A
:102E200005D03EF4909581959F4F089570956195DA
:102E30007F4F0895AA1BBB1B51E107C0AA1FBB1FF0
:102E4000A617B70710F0A61BB70B881F991F5A9536
:102E5000A9F780959095BC01CD010895EE0FFF1F55
:102E60000590F491E02D09940F931F93CF93DF9376
:102E70008230910510F482E090E0E091D102F0916F
:102E8000D20220E030E0A0E0B0E0309719F14081BC
:102E900051810281138148175907C8F0841795079B
:102EA00069F4109731F012960C93129713961C93B5
:102EB00027C00093D1021093D20222C02115310500
:102EC00019F04217530718F49A01BD01EF01DF0111
:102ED000F801DBCF21153105F9F0281B390B24301F
:102EE000310580F48A819B816115710521F0FB0118
:102EF0009383828304C09093D2028093D102FE0117
:102F0000329644C0FE01E20FF31F81939193225049
:102F10003109398328833AC02091CF023091D00201
:102F2000232B41F420910401309105013093D0020C
:102F30002093CF0220910201309103012115310528
:102F400041F42DB73EB74091060150910701241B73
:102F5000350BE091CF02F091D002E217F307A0F415
:102F60002E1B3F0B2817390778F0AC014E5F5F4FDF
:102F70002417350748F04E0F5F1F5093D00240933F
:102F8000CF028193919302C0E0E0F0E0CF01DF91A6
:102F9000CF911F910F910895CF93DF93009709F47C
:102FA00081C0FC01329713821282A091D102B091AC
:102FB000D202109781F420813181820F931F2091DA
:102FC000CF023091D0022817390751F5F093D00283
:102FD000E093CF0267C0ED0120E030E0CE17DF07BD
:102FE00040F44A815B819E0141155105F1F0EA01EF
:102FF000F5CFD383C28340815181840F951FC817B9
:10300000D90759F488819981840F951F029691837D
:1030100080838A819B81938382832115310529F4E2
:10302000F093D202E093D1023DC0E901FB83EA8331
:1030300049915991C40FD51FEC17FD0761F48081A8
:103040009181840F951F0296E9019983888382817B
:1030500093819B838A83E0E0F0E012968D919C91AE
:103060001397009719F0FD01DC01F7CF8D919C912A
:1030700011979D012E5F3F4F820F931F2091CF022A
:103080003091D0022817390769F4309729F410924B
:10309000D2021092D10202C013821282B093D002E7
:1030A000A093CF02DF91CF91089581E090E0F89452
:0830B0000C945A18F894FFCFAC
:1030B8000C000000D302800000000000680300102C
:1030C800111213141516171718191A1B1B1C1D1E7D
:1030D8001E1F2021222223242425262627282829AA
:1030E8002A2A2B2C2C2D2D2E2F2F303031313233F4
:1030F80033343435353636373738383839393A3A5B
:103108003B3B3B3C3C3D3D3D3E3E3F3F3F404040DE
:10311800404141414242424343434343444444447F
:10312800444545454545464646464646464646463E
:103138004747474747474747474747474747A59E62
:103148008C0000000047024402CD02D102C002B642
:1031580002AE02A002940250024A02550200000088
:103168000000000000380C380C380C380C380C38CB
:103178000C380C000000004205CB02F70041023E6B
:1031880002210216020C02030200000000F60600EB
:10319800000000D505000000000E080000000058DF
:1031A8000A000000009D0000000000260900000041
:1031B80000DD0A00000000380C00000000440CD9B3
:0C31C8000B070C910C8700160C2A0C0061
:00000001FF
